:020000040800F2
:1040000000C00020D17C00082D7C00082F7C000817
:10401000317C0008337C0008357C0008000000007B
:10402000000000000000000000000000377C0008D5
:10403000397C0008000000003B7C00083D7C000843
:10404000197D0008197D0008197D0008197D0008F8
:10405000197D0008197D0008417C0008197D0008C1
:10406000197D0008197D0008197D0008197D0008D8
:10407000197D0008197D0008197D0008497C000899
:10408000557C0008197D0008197D0008197D00087D
:10409000197D0008197D0008197D0008197D0008A8
:1040A000197D0008197D0008197D0008197D000898
:1040B000197D0008197D0008197D0008197D000888
:1040C000197D0008197D0008197D0008197D000878
:1040D000197D0008617C00086D7C0008197D0008CE
:1040E000197D0008197D0008197D0008197D000858
:1040F000197D0008197D0008197D0008197D000848
:10410000197D0008197D0008197D0008197D000837
:10411000197D0008197D0008797C0008197D0008C8
:10412000197D0008197D0008197D0008197D000817
:10413000000000000000000000000000000000007F
:10414000000000000000000000000000000000006F
:10415000000000000000000000000000000000005F
:10416000000000000000000000000000000000004F
:10417000000000000000000000000000000000003F
:10418000000000000000000000000000000000002F
:10419000000000000000000000000000000000001F
:1041A000000000000000000000000000000000000F
:1041B00000000000000000000000000000000000FF
:1041C00000000000000000000000000000000000EF
:1041D00000000000000000000000000000000000DF
:0441E0005FF8E0F1B3
:1041E40010B5054C237833B9044B13B10448AFF32D
:1041F40000800123237010BD78000020000000001F
:10420400448E000808B5034B1BB103490348AFF3C0
:10421400008008BD000000007C000020448E0008DF
:1042240038B50E4B054618784FF47A73B3FBF0F3A8
:104234000B4A1068B0FBF3F000F09EF8044658B93E
:104244000F2D09D8024629464FF0FF3000F054F8EC
:10425400044B20461D6038BD012038BD00000020FD
:104264001000002004000020074A08B5136803204A
:1042740043F01003136000F02DF80020FFF7D0FF87
:1042840003F0E2FB002008BD00200240034A044B77
:1042940011681B780B441360704700BFB005002001
:1042A40000000020014B1868704700BFB0050020D3
:1042B40038B50446FFF7F6FF0546631C1EBF044BE2
:1042C4001B78E418FFF7EEFF401B8442FAD838BD90
:1042D40000000020074A0002D36800F4E06023F4E1
:1042E400E0631B041B0C43F0BF6343F4003303433C
:1042F400D360704700ED00E0174B30B5DC68C4F3C1
:104304000224C4F10703251D042B28BF0423062D12
:104314004FF0010598BF002405FA03F303F1FF33BE
:1043240088BF033C1940A14005FA04F4013C224033
:10433400002842EA01024FEA0212AFBF00F16040D6
:10434400064B00F00F00D2B2A5BFD2B200F5614017
:104354001A5480F8002330BD00ED00E014ED00E0B5
:104364000123420900F01F0003FA00F0014B43F857
:104374002200704700E100E00138B0F1807F0AD2EA
:10438400F021064B064A586082F8231000200722C9
:1043940098601A6070470120704700BF10E000E089
:1043A40000ED00E010B5002832D00168194B142448
:1043B400994225D8184AA3F207430A44B2FBF4F2FF
:1043C400920002648468C36343680A682343C46830
:1043D40022F47F522343046922F0300223434469C8
:1043E400234384692343C469234313430B60012299
:1043F400002380F82120836380F82030184610BD04
:10440400064B0B44B3FBF4F39B000364044BD9E762
:10441400012010BD07040240F8FFFDBFF8FBFDBFFB
:1044240000040240F0B590F82040012C35D001245E
:1044340090F8215080F82040A5424FF000064FF03C
:10444400020428D180F82140046886632668076C3A
:1044540026F001062660C66BBD4075606360436844
:104464000568102BC36A0BBFA260A160E160E26023
:104474004BB1236843F00E0323602B68002043F004
:1044840001032B60F0BD236823F004032360236839
:1044940043F00A03F0E780F820600220F0BD00003A
:1044A40090F8213010B5022B03D00423836301203C
:1044B40010BD03681A6822F00E021A601A6822F00E
:1044C40001021A60294A934224D902F56272934286
:1044D40019D01432934218D01432934217D01432A4
:1044E40093420CBF4FF480534FF48033204A5360FF
:1044F4000123002480F82130436B80F820409BB3D3
:104504009847204610BD0123F0E71023EEE74FF44F
:104514008073EBE717498B4216D014318B4215D0C8
:1045240014318B4214D014318B4214D014318B4289
:1045340014D014318B4214D0934214BF4FF48033FF
:104544004FF080730C4AD2E70123FBE71023F9E70D
:104554004FF48073F6E74FF48053F3E74FF480335E
:10456400F0E74FF48013EDE7184610BD80000240D9
:1045740000040240080002400000024070B4042518
:10458400C66B026C3468036895402542196855D09F
:104594004D0753D51A6896065EBF1A6822F00402C6
:1045A4001A60604A93421FD902F56272934214D092
:1045B4001432934213D01432934212D014329342E1
:1045C4000CBF4FF480434FF48023574A5360C36AAF
:1045D400002B00F0A58070BC18470423F5E74023A6
:1045E400F3E74FF48063F0E750498B4216D014315F
:1045F4008B4215D014318B4214D014318B4214D019
:1046040014318B4214D014318B4214D0934214BF12
:104614004FF480234FF08063454AD7E70423FBE738
:104624004023F9E74FF48063F6E74FF48043F3E760
:104634004FF48023F0E74FF48003EDE70225954023
:10464400254257D08D0755D51A68940606D41A68A2
:1046540022F00A021A60012280F82120314A934292
:104664001ED902F56272934213D01432934212D0CF
:104674001432934211D0143293420CBF4FF40053BE
:104684004FF40033284A5360002380F82030836AB3
:104694009EE70223F6E72023F4E74FF40073F1E7E3
:1046A40022498B4216D014318B4215D014318B42DF
:1046B40014D014318B4214D014318B4214D01431E1
:1046C4008B4214D0934214BF4FF400334FF0007365
:1046D400174AD8E70223FBE72023F9E74FF40073D6
:1046E400F6E74FF40053F3E74FF40033F0E74FF4E9
:1046F4000013EDE708259540254211D009070FD591
:10470400196821F00E011960012303FA02F27260A4
:10471400836380F82130002380F82030036B57E74F
:1047240070BC704780000240000402400800024050
:10473400000002402DE9F74F002216466C4F6D4BE6
:10474400DFF8B8E1DFF8B8C14FF001080C6808FAE7
:1047540006F808EA0404A04540F085804D68122D4F
:1047640000F0B78000F28D80022D00F0AF8000F2DF
:104774008180002D00F09180012D00F0A5804FF084
:104784000F09FF2C93BF824606F18045083DD0F8FF
:1047940000B092BFB500D0F804B0AD0009FA05F836
:1047A4002BEA080802FA05F588BF00F1040A48EA72
:1047B4000505CAF80050D1F804A01AF0805F52D061
:1047C400BD6926F0030845F00105BD61BD6908F126
:1047D400804805F00105019508F5803806F0030BC3
:1047E400019D4FEA8B0BD8F8085009FA0BF925EA1A
:1047F4000909414DA84271D005F58065A8426FD0E2
:1048040005F58065A8426DD005F58065A8426BD09A
:1048140005F58065A84269D070450CBF05250625BD
:1048240005FA0BF545EA0905C8F808501D681AF49D
:10483400803F14BF2543A5431D605D681AF4003F03
:1048440014BF2543A5435D609D681AF4801F14BFFF
:104854002543A5439D60DD681AF4001F14BF2C4353
:1048640025EA0404DC600136102E7FF46DAF03B03A
:10487400BDE8F08F032D25D0112D80D1CA680432F4
:104884007DE7654509D012D8DFF878904D4504D00E
:1048940009F580394D457FF472AF8A68E2B1012A87
:1048A4000CBFC0F81080C0F81480082267E7DFF856
:1048B40058904D45F1D009F580394D45EDD0A9F515
:1048C4008019E7E700225AE7CA6858E7CA6808323D
:1048D40055E7CA680C3252E7042250E700259FE7E7
:1048E40001259DE702259BE7032599E7042597E722
:1048F400001002400004014000080140001C014077
:1049040000002110000011100000311083681942CA
:1049140014BF0120002070470AB1016170470904E7
:10492400FBE7C3685940C1607047704708B5044B42
:104934005969014202D05861FFF7F7FF08BD00BF73
:10494400000401400268536913F480630DD06FF4CE
:10495400806353610423202203640023036380F8EB
:104964003C3080F83D2001207047184670472DE9FF
:10497400F843044617469946C1F307488EB22568A2
:10498400B8F1010F0CBF6B69AB6936EA030314BFBE
:104994000120002008B9BDE8F8836B695A0512D5D7
:1049A4002B68202243F400732B606FF480636B61E7
:1049B4000423236400230120236384F83C3084F817
:1049C4003D20BDE8F8837B1CD9D04FB900232022B9
:1049D400236384F83C3084F83D200320BDE8F88349
:1049E400FFF760FCA0EB09008742C8D2EEE72DE98F
:1049F400F843044690461F46089EC1F307498DB20A
:104A04002368B9F1010F0CBF5B699B6935EA0303A5
:104A14000CBF01230023434502D00020BDE8F883E6
:104A24007B1CEDD05FB900232022236384F83C3043
:104A340084F83D20032084F83E30BDE8F883FFF776
:104A440031FC801B8742DBD2EDE770B504460D468E
:104A5400164623685B691B0601D5002070BD2046FD
:104A6400FFF770FFA8B96A1CF3D065B9236C202244
:104A740043F02003236400230320236384F83C30A1
:104A840084F83D2070BDFFF70DFC801B8542E0D209
:104A9400ECE7012070BD00002DE9FF4115460268D6
:104AA400984613680B9E43F4807313600F46009678
:104AB4000A9B00224FF001110446FFF798FF68B9E2
:104AC400236807F0FE071F610A9A33461A492046F5
:104AD400FFF74DFF30B1236C042B18D0032004B032
:104AE400BDE8F081236803905A690A9903929B698F
:104AF400324603932046039BFFF7A7FF48B1236C7C
:104B0400042BEBD12268136843F400731360012073
:104B1400E5E7B8F1010F236802D1EDB21D61DEE7CC
:104B24002A0A1A610A9932462046FFF78EFF0028A6
:104B3400E5D12368F1E700BF020001002DE9FF4140
:104B44009846036816461A680B9D42F480621A6000
:104B54001A680F4642F480721A604FF001110095F2
:104B64000A9B00220446FFF742FF80B92368FFB284
:104B740007F0FE021A612D492B460A9A2046FFF7D8
:104B8400F6FE40B1236C042B01D1012000E0032088
:104B940004B0BDE8F081236803905A690A9903922E
:104BA4009B692A4603932046039BFFF74EFF40B1BF
:104BB400236C042BEBD12268136843F40073136055
:104BC400E3E7B8F1010F236824D1F6B21E612A4647
:104BD4000A992046FFF739FF02460028E8D12168E8
:104BE40020460B6843F480730B6000950A9B4FF0DA
:104BF4000111FFF7FCFE0028C9D1236847F0010723
:104C04001F610A9A2B4609492046FFF7B0FE002887
:104C1400B8D1BDE7320A1A610A992A462046FFF73D
:104C240014FF0028C4D12368CFE700BF02000100AD
:104C340070B504460D4616462068436913F04003D8
:104C440001D0002070BD4269D2060BD56FF010026E
:104C540042612022236484F83C302363012084F8D9
:104C64003D2070BD5DB9236C032043F02003236411
:104C7400202384F83D30002384F83C3070BDFFF7D6
:104C840011FB801B8542D7D2EDE770B504460D4673
:104C9400164623685B695B0701D5002070BD20467A
:104CA400FFF750FEA8B96A1CF3D065B9236C202223
:104CB40043F02003236400230320236384F83C305F
:104CC40084F83D2070BDFFF7EDFA801B8542E0D2E9
:104CD400ECE7012070BD000038B5044608B9012096
:104CE40038BD90F83D3003F0FF021BB980F83C203A
:104CF40002F0CCFE2423226884F83D30136823F0AC
:104D04000103136000F0BAFC63682F4A934230D861
:104D14002E4A9042E3D92E4A2168B0FBF2F24A604F
:104D240001320A62284A0138934232D85B00B0FB50
:104D3400F3F0431CC3F30B03042B38BF0423CB61F0
:104D4400226AE369002013430B60E268236913437A
:104D54008B60A26963691343CB600B6843F0010362
:104D64000B602023206484F83D30206384F83E00E7
:104D740038BD184A9042B2D9154D4FF49672B0FB23
:104D8400F5F521686A434D604FF47A75B2FBF5F28C
:104D9400C6E7A26852B903EB4303B0FBF3F0431C2C
:104DA400C3F30B036BB143F40043C8E71922534325
:104DB400B0FBF3F0431CC3F30B0313B143F44043C0
:104DC400BDE70123BBE700BFA08601007F841E006E
:104DD40040420F00FF083D002DE9F34704469A4680
:104DE400884691460C9EFFF75DFA94F83D300546DF
:104DF400202B03D0022002B0BDE8F08700901923D5
:104E040001223E492046FFF7F2FD0028F2D194F832
:104E14003C30012BEED0012384F83C30236800277A
:104E24001A684146D20758BF1A6820465CBF42F050
:104E340001021A601A6822F400621A60212384F8BD
:104E44003D30402384F83E300A9B27646362BDF8FA
:104E54002C30019563852A4B0096E362638D4A46A4
:104E640023855346FFF718FE00282AD0236C84F8C4
:104E74003C70042B07D10120BDE7FFF7E6FD20B10C
:104E8400236C042B34D00320B5E7616A27684B1CDC
:104E940063620B78228D3B61638D501E013B9BB294
:104EA40063857B6980B25B0720850AD548B18B1C7A
:104EB40063624B78023A3B61638D2285013B9BB26E
:104EC4006385238D2A4631462046002BD5D1FFF732
:104ED400DCFE0028D4D12268136843F40073136005
:104EE400202384F83C0084F83D3084F83E0082E7B7
:104EF4002268136843F400731360BCE702001000D7
:104F04000000FFFF2DE9F047044686B09A460D469F
:104F14009146109FFFF7C6F994F83D300646202BC2
:104F240004D00225284606B0BDE8F0870090192376
:104F3400012281492046FFF75AFD0028F1D194F857
:104F44003C30012BEDD0012384F83C3023684FF032
:104F540000081A682946D20758BF1A6820465CBF61
:104F640042F001021A601A6822F400621A602223D5
:104F740084F83D30402384F83E300E9BC4F84080D2
:104F84006362BDF83C30019663856C4B0097E36225
:104F9400638D4A4623855346FFF7D0FD054630B15D
:104FA400236C84F83C80042B3DD10125BAE7228D83
:104FB400236892B902905A6902929A690292029AFB
:104FC4001A6842F400721A60202384F83D300023EA
:104FD40084F83E3084F83C30A4E7012A25D11A68CD
:104FE40022F480621A6072B6236803905A690392AD
:104FF4009A690392039A1A6842F400721A6062B6BC
:10500400DFF83C81238D002BDED0032B77D8012BD6
:1050140027D1324639462046FFF70AFE00283FD002
:10502400236C202BC1D103257CE7022A1A680ED1F8
:1050340042F400621A6072B6236804905A690492BA
:105044009A690492049A1A6822F48062D6E742F4B8
:1050540080621A6005905A6905929B690593059BC5
:10506400CEE7022B00963B464FF000024146204615
:1050740024D1FFF7BCFC0028D5D172B623681A6886
:1050840042F400721A60626A1B69511C61621370F7
:10509400238D013B2385638D013B9BB2638562B6FF
:1050A400636A5A1C6262226812691A70238D013B7A
:1050B4002385638D013B9BB26385A3E7FFF797FCD0
:1050C40002460028AFD121680B6823F480630B608B
:1050D40072B6636A2046591C6162216809691970B5
:1050E400238D0096013B2385638D4146013B9BB292
:1050F40063853B46FFF77BFC0028BFD093E732462D
:1051040039462046FFF794FD002889D1636A5A1C6A
:105114006262226812691A70238D2268013B23851A
:10512400638D013B9BB2638553695B077FF56AAF6F
:10513400636A591C6162B7E7020010000000FFFFB8
:105144000400010038B50446D8B14CF6CC420368DB
:105154001A6045F255521A6042685A6082689A6031
:10516400FFF7A0F805462368D86818B94AF6AA22BA
:105174001A6038BDFFF796F8401B3028F3D9032096
:1051840038BD012038BD000003682DE9F341DB0779
:10519400054610D42B689F075ED42B68190700F1CD
:1051A40095802B685A0700F1BF80EA69002A40F015
:1051B4002D81002014E0904C636803F00C03042B51
:1051C40007D0636803F00C03082B0CD16368DE037B
:1051D40009D523689C03DDD56B68002BDAD1012047
:1051E40002B0BDE8F0816B68B3F5803F10D123684D
:1051F40043F480332360FFF755F806462368980389
:10520400C8D4FFF74FF8801B6428F7D90320E7E7D9
:105214009BB9236823F480332360236823F4802319
:105224002360FFF73FF8064623689903B2D5FFF7DA
:1052340039F8801B6428F7D9E8E7B3F5A02F236871
:1052440003D143F480232360D1E723F48033236024
:10525400236823F48023CDE7674C636813F00C0FB5
:1052640007D0636803F00C03082B10D16368DA03DA
:105274000DD423689B0702D52B69012BAFD123687A
:105284006A6923F0F80343EAC203236085E72A69C5
:105294005A4B6AB101221A60FFF704F806462368E4
:1052A4009F07ECD4FEF7FEFF801B0228F7D9ADE779
:1052B4001A60FEF7F7FF0646236898077FF56DAF7F
:1052C400FEF7F0FF801B0228F6D99FE7AA694A4C33
:1052D4004B4BDAB101221A60FEF7E4FF0646636A1B
:1052E4009B070DD54FF4FA52464B1B68B3FBF2F300
:1052F400019300BF019B5A1E0192002BF9D150E784
:10530400FEF7D0FF801B0228E9D97FE71A60FEF779
:10531400C9FF0646636A9F077FF543AFFEF7C2FFE6
:10532400801B0228F6D971E7334CE369D80024D4F2
:105334000127E36943F08053E361E36903F0805399
:105344000093009B304E3368D90518D5EB68012BC8
:1053540026D1236A43F001032362FEF7A3FF41F23F
:1053640088368046236A9B073FD5002F3FF41DAF44
:10537400E36923F08053E36117E70027E2E733682A
:1053840043F480733360FEF78DFF80463368DA059B
:10539400DCD4FEF787FFA0EB08006428F6D935E7D4
:1053A400ABB9236A41F2883823F001032362236AEC
:1053B40023F004032362FEF775FF0646236A980769
:1053C400D3D5FEF76FFF801B4045F7D91EE7052BA9
:1053D400236A03D143F004032362BAE723F00103F1
:1053E4002362236A23F00403B6E7FEF75BFFA0EB16
:1053F4000800B042B6D909E700100240000042425A
:10540400800442421000002000700040224C636877
:1054140003F00C03082B3FF4E2AE00231F4E022AD4
:1054240033602BD1FEF73EFF0746236899011FD452
:105434002B6AB3F5803F05D16268A96822F4003273
:105444000A436260696A62680B4322F4741213436C
:10545400636001233360FEF725FF054623689A0144
:105464003FF5A7AEFEF71EFF401B0228F6D9CDE696
:10547400FEF718FFC01B0228D7D9C7E6FEF712FFB4
:10548400054623689B017FF594AEFEF70BFF401B96
:105494000228F6D9BAE600BF00100240600042427A
:1054A40030B5194B87B002AC03F1100522461868D9
:1054B4005968083303C2AB421446F7D101238DF86F
:1054C4000430022311498DF805304B6803F00C02B7
:1054D400082A17D1C3F3834206A80244DB0312F857
:1054E400102C0CD54B680A48C3F34043504306AA1A
:1054F400134413F8143CB0FBF3F007B030BD054877
:105504005043FAE70248F8E75C8E000800100240B6
:1055140000127A0000093D00544A2DE9F041136855
:10552400054603F007038B420E462AD329688C07ED
:1055340034D4CA0747D44D4A136803F007039E4284
:10554400C0F082802A684A4C12F0040F40F0878031
:10555400130706D563682A6923F4605343EAC20338
:105564006360FFF79DFF6368424AC3F30313D35C90
:10557400D840414B18600020FEF752FE0020BDE8E1
:10558400F081136823F007030B431360136803F0DF
:1055940007039942CAD00120BDE8F081344B11F0D1
:1055A400040F1EBF5A6842F4E0625A60080742BF03
:1055B4005A6842F460525A605A68A86822F0F002AD
:1055C40002435A60B5E76A68294C012A23681CD152
:1055D40013F4003FDFD0636841F2883823F00303FB
:1055E40013436360FEF75EFE6B680746012B14D11C
:1055F400636803F00C03042B9DD0FEF753FEC01B1D
:105604004045F5D90320BDE8F081022A02D113F008
:10561400007FDFE713F0020FDCE7022B0FD1636892
:1056240003F00C03082B86D0FEF73CFEC01B40455C
:10563400F5D9E7E7FEF736FEC01B4045E2D86368BC
:1056440013F00C0FF6D176E7136823F00703334306
:105654001360136803F007039E429CD172E76368EA
:10566400E96823F4E0630B43636071E700200240C0
:1056740000100240C090000810000020044B054AAE
:105684005B68C3F30223D35C034A1068D8407047B5
:1056940000100240D090000810000020044B054A7E
:1056A4005B68C3F3C223D35C034A1068D8407047D5
:1056B40000100240D0900008100000200368002071
:1056C400DA6842F00102DA601A6842F001021A60F4
:1056D40070477047704770477047036810B51A6980
:1056E400044691070ED5DA6892070BD56FF00202D3
:1056F4001A6101229B6902779B0777D0FFF7EAFFC3
:105704000023237723681A69500710D5DA685107F4
:105714000DD56FF004021A6102229B69227713F4FB
:10572400407F204668D0FFF7D5FF00232377236806
:105734001A6912070FD5DA6810070CD56FF0080242
:105744001A610422DB692277990720465AD0FFF7B1
:10575400C1FF0023237723681A69D20610D5DA68BB
:10576400D0060DD56FF010021A610822DB6922778A
:1057740013F4407F20464BD0FFF7ACFF0023237780
:1057840023681A69D10708D5DA68D20705D56FF0FE
:10579400010220461A6101F02FFC23681A691006E1
:1057A40008D5DA68110605D56FF0800220461A6123
:1057B40000F0BFF823681A69520608D5DA68500663
:1057C40005D56FF0400220461A61FFF785FF236874
:1057D4001A69910622D5DA6892061FD56FF0200265
:1057E4002046BDE810401A6100F0A2B8FFF771FF2F
:1057F4002046FFF770FF83E7FFF76BFF2046FFF7B4
:105804006AFF92E7FFF765FF2046FFF764FFA0E712
:10581400FFF75FFF2046FFF75EFFAFE710BD000014
:10582400244A0368904212D002F5006290420ED0DE
:10583400B0F1804F0BD0A2F59832904207D002F518
:105844008062904203D002F5806290421DD14A6882
:1058540023F070031343174A904212D002F50062FA
:1058640090420ED0B0F1804F0BD0A2F59832904206
:1058740007D002F58062904203D002F58062904224
:1058840003D1CA6823F4407313434A6923F08003A5
:10589400134303608B68C3620B688362054B9842B1
:1058A40003D003F50063984201D10B69036301231C
:1058B40043617047002C014010B50446A0B190F834
:1058C4003D3003F0FF021BB980F83C2002F010F9D0
:1058D4000223206884F83D30211DFFF7A1FF012336
:1058E400002084F83D3010BD012010BD90F83C30FC
:1058F40010B5012B4FF0020318D080F83D30036837
:105904000C685A68496822F070025A605A68224347
:105914005A609A6822F080029A609A680A439A60F0
:10592400012380F83D30002380F83C30184610BD38
:10593400704770470368DA6822F49072DA605A6933
:1059440022F001025A61202380F83A3070470000A7
:105954002DE9F0470568C2682B69016923F44053B7
:1059640013432B618368EA680B43416922F4B05204
:1059740022F00C020B431343EB606B69826923F43E
:10598400407313436B61404B81469D424FF01904B1
:1059940046D1FFF783FE04FB00F3D9F804604FF00F
:1059A4006408B600B3FBF6F3B3FBF8F31E01FFF78C
:1059B40075FE6043D9F804309B00B0FBF3F7FFF7A2
:1059C4006DFE6043D9F804309B00B0FBF3F3B3FBE6
:1059D400F8F308FB13731B013233B3FBF8F303F042
:1059E400F007FFF75BFE6043D9F804209200B0FB98
:1059F400F2FAFFF753FE6043D9F804309B00B0FB82
:105A0400F3F3B3FBF8F308FB13A31B013233B3FB2B
:105A1400F8F303F00F033B433344AB60BDE8F08776
:105A2400FFF72CFE04FB00F3D9F804604FF0640880
:105A3400B600B3FBF6F3B3FBF8F31E01FFF71EFE4B
:105A44006043D9F804309B00B0FBF3F7FFF716FE70
:105A54006043D9F804309B00B0FBF3F3B3FBF8F3D5
:105A640008FB13731B013233B3FBF8F303F0F007A5
:105A7400FFF704FE6043D9F804209200B0FBF2FA69
:105A8400FFF7FCFDB7E700BF00380140F8B5044656
:105A94000E4617461D4621680B6836EA030301D1FA
:105AA4000020F8BD6B1CF7D095B923680320DA6891
:105AB40022F4D072DA605A6922F001025A6120237A
:105AC40084F8393084F83A30002384F83830F8BD4B
:105AD400FEF7E8FBC01B8542DDD2E6E710B50446BD
:105AE40040B390F8393003F0FF021BB980F8382036
:105AF40002F012F82423226884F83930D36820464F
:105B040023F40053D360FFF723FF236800201A69AE
:105B140022F490421A615A6922F02A025A61DA6820
:105B240042F40052DA602023E06384F8393084F8C8
:105B34003A3010BD012010BD2DE9F0411F4690F808
:105B440039300446202B0D4690464ED1002949D0C9
:105B5400002A47D090F83830012B46D0012380F832
:105B640038300023C363212380F83930FEF79AFBD1
:105B74000646A4F82480A4F82680E38C9BB26BB973
:105B84003B46324640212046FFF780FFA8B9202338
:105B940084F8380084F83930BDE8F081E38C32466B
:105BA400013B9BB2E384A3688021B3F5805F204668
:105BB4003B460ED1FFF76AFF10B10320BDE8F08128
:105BC4002B882268C3F308035360236943B9023561
:105BD400D3E7FFF75BFF0028EFD123682A785A60E8
:105BE4000135CAE70120BDE8F0810220BDE8F0815B
:105BF400134690F83A2073B5202A054638D1002977
:105C040034D0002B32D090F83820012A30D0012231
:105C1400002480F83820222281628385C46380F8BE
:105C24003A20406B134A2E688262134A4463C2626C
:105C3400124A02630A46311DFEF7F4FB20462B6824
:105C440001941A6801925A6885F838400192019AC1
:105C5400DA6842F48072DA605A6942F001025A61E9
:105C64005A6942F040025A6102B070BD0120FBE75C
:105C74000220F9E7875C00083D5D0008495D0008E3
:105C8400704708B50368426A1B6813F0200310D1FB
:105C9400D3851368D96821F48071D960596921F0DA
:105CA40001015961596921F040015961202382F8A9
:105CB4003A30104601F06EF908BD90F83A3010B54C
:105CC400222B36D183680169B3F5805F0268836A49
:105CD40023D15268E9B9C2F3080223F8022B836284
:105CE400C48D013CA4B2C4858CB90368DA6822F07F
:105CF4002002DA60DA6822F48072DA605A6922F0EB
:105D040001025A61202380F83A3001F043F900205F
:105D140010BDD2B223F8012BE1E721B9591C526816
:105D240081621A70DCE75268591C816202F07F02BA
:105D3400F7E7022010BD704708B5406AFFF7FBFF84
:105D440008BD7047416A08B50B685A6991F8390073
:105D540021280AD1120608D50022CA84DA6822F062
:105D6400C002DA60202281F839205B6991F83A2078
:105D7400222A06D15B0604D500230846CB85FFF70B
:105D8400D9FDCB6B084643F01003CB63FFF7D9FF73
:105D940008BD0000036870B51A6804461607D96880
:105DA4005D6907D196065AD58D0658D5BDE8704071
:105DB400FFF783BF15F0010502D111F4907F4ED097
:105DC400D30705D5CE0542BFE36B43F00103E3637C
:105DD400500704D51DB1E36B43F00203E36393075B
:105DE40004D51DB1E36B43F00403E363160704D544
:105DF4001DB1E36B43F00803E363E36B002B66D050
:105E0400950604D5880602D52046FFF756FF236879
:105E140020465D69E26B110702D415F040051AD0E3
:105E2400FFF788FD23685A69520610D55A69606BDA
:105E340022F040025A6150B1254B4363FEF730FB18
:105E4400002844D0606BBDE87040436B184720467F
:105E5400FFF777FF70BDFFF774FFE56370BD1606AB
:105E640027D50D0625D594F83920212A2FD1A268EB
:105E7400B2F5805F226A17D11188C1F30801596015
:105E8400216979B902322262E28C013A92B2E28447
:105E9400EAB9DA6822F08002DA60DA6842F0400295
:105EA400DA6070BD0132EEE7511C216212785A604B
:105EB400EAE750060BD54A0609D5DA68204622F0EF
:105EC4004002DA60202384F83930FFF7D9FE70BD30
:105ED400D95E000808B50023406AC385C384FFF770
:105EE40030FF08BD002382B00093009B834201DB96
:105EF40002B07047019B01330193009B0133F3E728
:105F040070B505460824144E0420FFF7EBFF002269
:105F140008213046FEF700FD2B064CBF012200226B
:105F240020213046FEF7F8FC0420FFF7DBFF0122B6
:105F340008213046FEF7F0FC013C04206D00FFF719
:105F4400D1FF14F0FF04EDB2DED12246BDE870406B
:105F540008210148FEF7E0BC000C014070B508259B
:105F64000024104E0420FFF7BDFF08213046012213
:105F7400FEF7D2FC640010213046E4B2FEF7C6FC02
:105F840008B144F001040420FFF7ACFF013D0022F6
:105F940008213046FEF7C0FC15F0FF05E2D120468B
:105FA40070BD00BF000C0140FFF7AABF2DE9F04F00
:105FB40006460F4690461D4600244FF4FA694FF0FA
:105FC400010ADFF840B087B0AC4202D107B0BDE8A7
:105FD400F08F3B1908EB0402009392B21023A02126
:105FE400CDF80890CDF804A03046FEF7F5FE0590F4
:105FF4000520FEF75DF9059B13B1584601F038FF03
:106004000134E1E76C8E00087FB5002206AB03F88B
:10601400042D4FF4FA62029201220093019210239C
:106024000A46A121FEF76EFF9DF8140007B05DF843
:1060340004FB0000BFF34F8F0549064BCA6802F406
:10604400E0621343CB60BFF34F8F00BFFDE700BF97
:1060540000ED00E00400FA050138C0B207289ABF39
:10606400014B185C00207047828E00080138C0B2D2
:1060740007289ABF024B33F810000020704700BF76
:106084008A8E00082DE9F74F00216848684EFFF713
:10609400BBFF0124B046674D644F28702146384643
:1060A400FFF7B2FF611C0002708089B23846FFF727
:1060B400ABFF06347388A4B21843312C26F8020FC0
:1060C400ECD1DFF89C9103244F46584E21463046CC
:1060D400FFF79AFF611C0002A9F8020089B230465A
:1060E400FFF792FF0634B9F80230A4B21843332CF8
:1060F40029F8020FEAD1DFF86C910524CB464B4E08
:1061040021463046FFF780FF611C0002A9F8020017
:1061140089B23046FFF778FF0634B9F80230A4B2EA
:106124001843352C29F8020FEAD100244FF0320924
:10613400661CF0B2FFF79AFF4FF0000A024609FB13
:1061440004F402EB0A0189B238480192FFF75CFFBC
:10615400394B0AEB04010AF1010A1944BAF1320F6E
:1061640081F83200019AECD1082E3446E0D1297826
:10617400324801F009FE0124DFF8EC90304E314D35
:1061840038F814202146484601F0FEFD37F8142063
:106194002146304601F0F8FD3BF8142021462846FC
:1061A400013401F0F1FD092CEAD14FF4E1711F48EB
:1061B400FFF72AFFFF2835D04FF4E1711B48FFF7A2
:1061C40023FF214C40F2C31120701848FFF71CFF35
:1061D4004FF4E27160711548FFF716FF40F2C511E4
:1061E400A0701248FFF710FF4FF4E371E0700F48FE
:1061F400FFF70AFF21782071144801F0C5FD617989
:10620400134801F0C1FDA178124801F0BDFDE17809
:10621400114801F0B9FD2179104803B0BDE8F04FF1
:1062240001F0B2BD03B0BDE8F08F00BF0C06002042
:106234009C0300200004002002010020B78E000807
:10624400EC8E0008138F0008080000203A8F000825
:10625400548F00086E8F0008888F0008A28F0008F2
:106264008A030020C4020020C58E00082DE9F341F2
:1062740043780446013B172B16D8DFE803F0380CAB
:1062840038151B2C38383D15151515414A2515258B
:106294001515157181250A2100F0E2FE0123002263
:1062A4004D494E48FFF782FE00224D4B1A6002B062
:1062B400BDE8F0811425C078A2784A4B0332214608
:1062C40005FB003001F04CFDA17820460331C9B232
:1062D40000F0C6FEE8E781780331C9B200F0C0FEE1
:1062E400A07AFFF7B9FE06230246211DD9E707214C
:1062F400204600F0ADFED7E781780331C9B2F7E755
:10630400C078FFF7B3FEA37802460333DBB221461D
:10631400C7E7807AFFF7AAFE811C89B22F48FFF7EE
:1063240073FEA070E078FFF7A1FE00230746DFF8B4
:10633400AC80A178DEB25D1C8B1CB34208DA204627
:106344000F2300F8013F4D1C01F045FB6055BBE7EE
:10635400B91989B24046FFF757FE2B46A055E8E726
:10636400827801460332684601F0FAFC1A4B9DF824
:1063740004201B789A429AD1012000F05DFE93E735
:106384001823194D43700379C1786B7143792970CF
:10639400AB708379EB70C37914482B7101F0F4FC72
:1063A4006979134801F0F0FCA978124801F0ECFC7B
:1063B400E978114801F0E8FC2979104801F0E4FC7F
:1063C400A3784FF4E172023BDBB2E11C0348FFF710
:1063D400EDFDFFF72FFE00BF000400200C06002097
:1063E400F8030020D6020020080000203A8F00089D
:1063F400548F00086E8F0008888F0008A28F000851
:1064040008B5082850D8DFE800F00530383C40448F
:10641400484B2C0000224FF480612448FEF77CFA9C
:1064240000224FF400612148FEF776FA00224FF46F
:1064340080511E48FEF770FA002204211C48FEF722
:106444006BFA002240211B48FEF766FA00228021E5
:106454001848FEF761FA00224FF480711548FEF7E0
:106464005BFA00224FF4007115E000224FF48061C2
:106474000E48BDE80840FEF74FBA00224FF4006111
:10648400F6E700224FF48051F2E700220421084885
:10649400EFE7002240210748EBE700228021FAE7DA
:1064A40000224FF48071F6E708BD00BF00100140E0
:1064B40000140140000C014008B5082850D8DFE85A
:1064C40000F00530383C4044484B2C0001224FF486
:1064D40080612448FEF720FA01224FF4006121482C
:1064E400FEF71AFA01224FF480511E48FEF714FAFF
:1064F400012204211C48FEF70FFA012240211B4807
:10650400FEF70AFA012280211848FEF705FA012253
:106514004FF480711548FEF7FFF901224FF4007122
:1065240015E001224FF480610E48BDE80840FEF7F3
:10653400F3B901224FF40061F6E701224FF48051D0
:10654400F2E7012204210848EFE70122402107482D
:10655400EBE701228021FAE701224FF48071F6E78C
:1065640008BD00BF0010014000140140000C0140B0
:106574002DE9F04700252C46DFF86090DFF86080B5
:10658400DFF860A099F80030EFB2BB420BD20CBB2D
:10659400224611484FF48051FEF7BEF92046BDE86B
:1065A400F047FFF789BF18F807001AF80060012EBA
:1065B4000CD1094832464FF48051FEF7ADF918F872
:1065C4000700FFF71DFF01353446DBE7FFF774FFD3
:1065D4002646F8E7BDE8F087000C0140AE03002032
:1065E400AF03002094000020002230B5104601259E
:1065F400074B084C1978D3B2994200D830BD135DCB
:1066040023B1013B05FA03F31843C0B20132F2E7A8
:10661400AE030020AF0300200138C0B207289ABFA0
:10662400014B185C002070479A8E0008F8B5BE2311
:106634001D4C00222370EB236260E3711623637008
:106644000523A370194B1A4E1B7805463078E37066
:10665400FFF7E2FFC8B1174B4FF0010E1F78134646
:106664002179D8B2B84215D902B121710023EA5C6C
:1066740061799A4001330A43082B6271F7D10521ED
:106684000D4801F0A8F9A071F8BD0C48BDE8F84028
:1066940001F0EEBB325C0133013A0EFA02F211430F
:1066A400C9B20122DDE700BF9D00002000040020E4
:1066B400AF030020AE0300209E000020BC8F000822
:1066C4002DE9F74F8179C279C378264E42EA012237
:1066D400047A26F81320427A234942EA042221F854
:1066E4001320847AC27A214D42EA042225F8132029
:1066F40000224FF0010E144691461D4B284693F894
:1067040000C01C4F1C4DDFF884800191D3B2634557
:106714000AD91A48FFF78AFF194B1A78A24218BF00
:106724001C7003B0BDE8F08F1649CB5C37F813B08A
:1067340036F813A0D3450DD8134931F813B0019995
:1067440031F813A0D34505D838F813B030F813A0A6
:10675400D34504D9012405F803E00132D6E705F84E
:106764000390FAE7DC030020CA030020B8030020EA
:10677400AE0300209C03002094000020950000201C
:1067840001010020AF0300208A030020C40200207E
:1067940030B545789BB004466422002101A801F07D
:1067A400EAFA6B1E172B35D8DFE813F0180039000E
:1067B4004300550063009500340034003400BC00ED
:1067C400340034003400BE00C500CC003400E300C3
:1067D40034003400120134001C012B019A4A9B48F6
:1067E40011784B1C415CDBB2217199491370097813
:1067F400601C994238BF0023A17838BF137001F0A0
:10680400EAF86071A2882068A3790190ADF80820A5
:106814008DF80A3001A8FFF729FD1BB030BDA2781E
:106824002146033201A801F09BFAE278894B1A70E1
:10683400F0E7012000F006FCA2782146033201A80B
:1068440001F08EFA9DF806100DF1050001F0C3F871
:106854008DF80900DEE7E1780029DED07E4801F0FA
:1068640093FA7B4A1378591C1170E178774AD15412
:10687400D0E70021E378794A2046D154A378013344
:10688400A370FFF71DFFA2782146033201A801F08F
:1068940067FAFFF7A9FE9DF806301AAA134403F815
:1068A400650C9DF806300DF1050013446C4A5279CD
:1068B40003F8642C9DF80640214601F08CF81AABCD
:1068C4001C4404F8630C9DF806301AAA1344EB2206
:1068D40003F8622C9EE7A2782146033201A801F056
:1068E4003FFA22796379A17A43EA02235D4A0DF1E2
:1068F400050022F81130A279E379A17A43EA022350
:10690400594A22F81130227A637AA17A43EA02239F
:10691400564A22F811309DF8061001F05CF88DF803
:106924000F0077E7FFF786FBA2782146033201A820
:1069340001F016FA6EE70F238DF80530E3788DF831
:10694400073067E7BE238DF80430102303218DF848
:106954000530404B0DF105001B788DF806108DF8BD
:10696400073001F038F8EB238DF808008DF8093072
:1069740050E7BE238DF80430122308218DF805302A
:10698400384AE3788DF8061032F8132022FA01F021
:106994008DF80820344A8DF8070032F8132022FAC3
:1069A40001F08DF80A20314A8DF8090032F81330CD
:1069B4000DF1050023FA01F28DF80C308DF80B204F
:1069C40001F009F8EB238DF80D008DF80E3021E766
:1069D400A2782146033201A801F0C2F916238DF8EA
:1069E400053017E7A578214603352A4601A801F0AA
:1069F400B7F99DF806100DF1050000F0ECFF6055A5
:106A040008E7BE238DF80430182307218DF80530DC
:106A1400174B0DF105001A798DF806108DF8072033
:106A24005A7A8DF808209A798DF80920DA791B7A38
:106A34008DF80A208DF80B3000F0CDFFEB238DF894
:106A44000C008DF80D30E5E6F7030020AF030020BD
:106A5400AE03002000040020A28E0008EE030020F4
:106A64009D0000209C0300208A030020C402002013
:106A74001C090020BFF34F8F0549064BCA6802F476
:106A8400E0621343CB60BFF34F8F00BFFDE700BF4D
:106A940000ED00E00400FA054B1E5A42018A5A41F7
:106AA4004069FDF739BF10B504460121FFF7F4FF33
:106AB400218860680122BDE81040FDF72DBF10B5A4
:106AC4000C460021FFF7E8FF2046BDE81040FFF721
:106AD4006BBAF8B50E4604461F46002100681546F9
:106AE400FFF7DAFF46F080012068FFF7E8FF013F77
:106AF4006E1E3D44AE4204D101212068FFF7CCFF55
:106B0400F8BD16F8011F2068FFF7D9FFF2E708B5B2
:106B14000021FFF7C1FFFFF721FAC0B208BDFDF75E
:106B2400C7BB08B50189C068FDF7F0FE431E584293
:106B3400584108BD38B504460068FFF7C0FF206817
:106B4400FFF7E5FF054601212068FFF7A5FF28466A
:106B540038BD70B504460E46154600210068FFF79F
:106B64009BFF46F080012068FFF7A9FF29462068B3
:106B7400FFF7A5FF01212068FFF78EFF70BD012BF1
:106B8400F8B505460F4616461C4616D9002100687E
:106B9400FFF782FF39462868FFF791FF013CE4B212
:106BA400771E34442868FFF7B2FF07F8010FA742A5
:106BB400F8D101212868FFF76FFFF8BD012B01D937
:106BC400FFF787BF70474279437A02F00F0242F021
:106BD400700242EAC312D2B20921FFF7BABF0122FE
:106BE40010B511460446FFF7B4FF0123E37210BD4C
:106BF40010B5802201210446FFF7ABFF0023E372A6
:106C040010BD80220121FFF7A4BF00002DE9F84345
:106C140004460D4691461F469DF820609DF8248049
:106C2400FFF7E6FF0F20FFF77AFF2046FFF7E9FFA3
:106C3400344A05EB45052A44032306212046FFF781
:106C440048FF314B092113F809202046FFF781FF43
:106C54000B2220461146FFF77CFF2046FFF7B3FFC7
:106C640042460C212046FFF774FF284BDD5D284B7C
:106C7400062D9A5D4FEA021237D10332D2B21D219A
:106C84002046FFF766FF67221E212046FFF761FFBB
:106C940031212046FFF74EFF00F0F80242F00502D2
:106CA40031212046FFF755FF0C2237212046FFF7FC
:106CB40050FF2046FF221F21FFF74BFF20460022F2
:106CC4002021FFF746FF20460C222121FFF741FF38
:106CD400204601224121FFF73CFF0023204684F88F
:106CE4000C31BDE8F843FFF77ABF023202F0FE022E
:106CF4001D212046FFF72DFF2A010732D2B21E21A3
:106D0400D4E700BFCE8F00081F900008239000082E
:106D1400F88F000830B5457A85B00295C479057AB4
:106D240083794279017901950094FFF76FFF05B0EB
:106D340030BDFF221221FFF70CBF000070B50446DE
:106D44000E46A1721546FFF7E5FF84224D21204629
:106D5400FFF7FFFEFF2224212046FFF7FAFE01225F
:106D640040212046FFF7F5FE3F2211212046FFF780
:106D7400F0FE2046FFF7DDFF324622212046FFF7D2
:106D8400E8FE0F212046FFF7D5FE0D2102462046DE
:106D9400FFF7DFFE852201212046FFF7DAFE0023FC
:106DA40084F80C3118212046FFF7C4FE43070DD4A4
:106DB400013D07D14FF4A3720649074800F0E4FFF0
:106DC400FFF758FE0120FFF7AAFEEBE7032301209B
:106DD400E37270BD2A9000080290000870B5044662
:106DE4000068FFF79EFEF0B104F10C064FF48072C8
:106DF4000021304600F0BFFF10212046FFF79AFE25
:106E04000D2102462046FFF7A4FEA37973B9A57AA3
:106E140020462B4632460021FFF7B1FE84F80C5180
:106E24002046FFF786FF94F80C0170BD132120461D
:106E3400FFF780FE0546EBE770B504460E46A172E7
:106E44001546FFF767FF87224D212046FFF781FE95
:106E5400002224212046FFF77CFE412240212046C7
:106E6400FFF777FE2046FFF764FFF7221121204643
:106E7400FFF76FFE324622212046FFF76AFE0E21FD
:106E84002046FFF757FE0D2102462046FFF761FE1C
:106E940022212046FFF74EFE864209D0013DF7D15C
:106EA40040F283120449054800F06EFFFFF7E2FD4B
:106EB40002230120E37270BD3D9000080290000897
:106EC40038B504461D4613460A460021FFF776FEF0
:106ED400832201212046FFF73CFE2068FFF721FEB4
:106EE40068B9013D07D14FF4CE720B490B4800F04D
:106EF4004BFFFFF7BFFD0120FFF711FEEDE7122165
:106F04002046FFF717FE2046FFF713FF2046FFF742
:106F140066FE012038BD00BF5090000802900008B2
:106F24002DE9F84F04468B46924699469DF82880F1
:106F34009DF82C709DF830609DF834500068FFF780
:106F4400B2FD84F804B084F805A084F8069084F8AF
:106F54000780A772267265722046BDE8F84FFFF7D6
:106F6400D9BE70B50E4690F80C41054600F10C01EF
:106F74002246304600F0F4FE0023335585F80C31E8
:106F8400204670BD08B51B21FFF7D4FD0A38C0B2F6
:106F940008BD00000268104B10B59A420BD10F4A8D
:106FA4000F4913780C780F49CC540133DBB2632BAF
:106FB40088BF0023137002680B4B9A420BD10B4A13
:106FC4000B49137808780B49C8540133DBB2632B9F
:106FD40088BF0023137010BD00380140D604002080
:106FE400340800200C04002000440040D704002092
:106FF400600600207004002002680A4B9A420FD1F8
:10700400094A136801331360084A13680133136093
:10701400074A136801331360064A13680133136087
:10702400704700BF00100040040400200804002042
:10703400F8030020FC030020014B1870704700BFC8
:10704400E4060020014B1870704700BF01040020C3
:107054000A460A2301460148FEF76EBDD8080020FF
:107064000A460A2301460148FEF766BD2C070020A4
:1070740010B514460A230248FEF75EFD204610BDF3
:107084002C070020F8B50D468178044643185A7839
:10709400013000F0BBFCC8B9114F2B78461CC0B2BC
:1070A40083420DD8A378002123445A780D4800F078
:1070B4006BFE2046BDE8F8406422002100F05BBE70
:1070C400215C384600F060FE3046E6E7012803D133
:1070D4002046FFF75DFBECE7034800F0C9FEE8E754
:1070E40070900008769000089C900008BE2313B5A9
:1070F40002218DF80030192304460DF101008DF8AA
:1071040001308DF8021000F066FCEB238DF80300CB
:107114008DF80430082C44D8DFE804F0CA05454D46
:107124005B6F88A6CA009DF8021068460331C9B295
:10713400FFF796FF00224FF400517248FDF7ECFB75
:107144006420FDF7B5F801224FF400516D48FDF7B6
:10715400E3FB00224FF480416A48FDF7DDFB002287
:107164004FF400416748FDF7D7FB002240216648F1
:10717400FDF7D2FB002280216348FDF7CDFB0022FE
:107184004FF480716048FDF7C7FB00224FF4007193
:107194005D48FDF7C1FB00224FF480715B48FDF7A9
:1071A400BBFB02B010BD01224FF400515548FDF75E
:1071B400B3FB0122CEE701224FF400515148FDF701
:1071C400ABFB01224FF480414E48FDF7A5FB0122A1
:1071D400C6E701224FF400514A48FDF79DFB012206
:1071E4004FF480414748FDF797FB01224FF40041DB
:1071F4004448FDF791FB0122B8E701224FF4005106
:107204004048FDF789FB01224FF480413D48FDF7DA
:1072140083FB01224FF400413A48FDF77DFB012234
:1072240040213948FDF778FB0122A4E701224FF4FD
:1072340000513448FDF770FB01224FF4804131487E
:10724400FDF76AFB01224FF400412E48FDF764FB71
:10725400012240212C48FDF75FFB012280212A48AE
:10726400FDF75AFB01228BE701224FF40051254818
:10727400FDF752FB01224FF480412248FDF74CFBFD
:1072840001224FF400411F48FDF746FB0122402133
:107294001D48FDF741FB012280211B48FDF73CFB03
:1072A40001224FF480711848FDF736FB01226DE787
:1072B40001224FF400511348FDF72EFB01224FF435
:1072C40080411048FDF728FB01224FF400410D488E
:1072D400FDF722FB012240210B48FDF71DFB012293
:1072E40080210948FDF718FB01224FF480710648FC
:1072F400FDF712FB01224FF400710348FDF70CFB6C
:10730400012249E7000C014000100140000801403F
:107314001021164B164A30B5DA605A614FF4004218
:107324009960012113481A614579134C134A85B0B9
:1073340083E8060023604278837801780395057911
:1073440002950A250195C07800902046FFF7E8FDD4
:1073540000220B4B08211A6020464FF4FA62FFF713
:10736400EDFC084B186005B030BD00BFC806002016
:1073740000080140080000201C090020000C014006
:107384002C0A0020180900202DE9F041254B1F7814
:10739400002F44D1244E254C3378012B28D1244B83
:1073A4001A78BE2A24D11A68224D99782A60DFF807
:1073B40090805A6803316A60C8F800104FF4FA628A
:1073C400C9B21D48FFF738FD4FF4FA63206098F8FE
:1073D400002029461848FFF773FD4FF4FA62206035
:1073E400082115483770FFF7A9FC2060BDE8F0813B
:1073F4001148FFF7F3FC0246206080B10D490E48A6
:10740400FFF7AFFD0C48FFF7BDFD01460B4800F048
:10741400BBFCBDE8F04105490648FFF733BEBDE8B3
:10742400F08100BF01040020E406002018090020B8
:107434009D0000206C0700201C09002064900008B7
:10744400F805002070B5304A304B11781B78304C69
:107454008B4213D02F4B1878451C1D704B1CDBB28C
:107464001370632B4FF0000388BF13702A4A2B4D0F
:10747400136001236D5C2A4923700D54294A2A4B59
:1074840011781B788B4213D0284B1878451C1D703B
:107494004B1CDBB21370632B4FF0000388BF1370D7
:1074A400234A244D136002236D5C234923700D5439
:1074B4002278224D012A2A7010D1174B1B68642BA5
:1074C4000CD90026134B114915481E70FFF7DAFD3D
:1074D40064223146124800F04EFC26702B78022BB1
:1074E40010D1134B1B68642B0CD900250F4B0E498C
:1074F40011481D70FFF7C6FD642229460E4800F0AE
:107504003AFC257070BD00BFD8040020D6040020CA
:10751400FC050020D4040020040400200C040020F6
:10752400DA040020D9040020D7040020D504002068
:1075340008040020700400203E050020A20500205D
:1075440003232DE9F0410425BE27DFF8188186B016
:107554008DF809303C4C98F8003029468DF80B30F2
:1075640023780DF109008DF80C308DF808708DF832
:107574000A5000F030FAEB261A2302218DF80D0090
:107584000DF101008DF801308DF802108DF80E60B8
:107594008DF8007000F01FFA01238DF8113098F86F
:1075A40000308DF803008DF81330237829460DF14F
:1075B40011008DF814308DF804608DF810708DF87A
:1075C400125000F008FA214B8DF815001B688DF855
:1075D4001660B3F5FA7F28D91D4B1A78012A30D1E9
:1075E400207820B91B4A106050601B4A107001308B
:1075F400C0B2082820708DF80C0019D9002528463F
:107604001D70FFF773FD9DF8021068460331C9B27F
:107614002570FFF725FD4AF6AA22104B4FF40041CE
:107624001B680F481A60FDF77CF906B0BDE8F081CD
:10763400FFF75CFD6420FCF73BFE02A8FFF7A8F807
:10764400E9E704A8FAE700BF02040020F8030020D9
:1076540001040020AF030020AE0300200006002038
:107664000010014000040020054B5B6A9B0005D517
:107674000122044B04481A6000F0FABB704700BFB3
:1076840000100240E0044242AA90000810B590B0F5
:107694002822002106A800F06EFB0021142201A874
:1076A40000F069FB09230122069302244FF480337E
:1076B40006A807930A920C920E930D94FDF764FDAD
:1076C4000F23002101934FF4806301A802940391D6
:1076D40004930591FDF720FF10B010BDBE232DE9E2
:1076E40080488DB002268DF81830192331460DEBF1
:1076F40003004FF010098DF819308DF81A6000F06E
:107704006AF9EB239E4D8DF81C308DF81B00FCF7B5
:10771400ABFDFFF7BBFF4A46002108A800F02BFB96
:10772400AB69002243EA0903AB61AB6949F6F07126
:1077340003EA09030293029BAB69924843F02003D6
:10774400AB61AB69002403F020030393039BAB6993
:10775400012743F00403AB61AB69DFF8708203F0E7
:1077640004030493049BAB694FF00C0A43F0080331
:10777400AB61AB694FF4E13B03F008030593059B50
:10778400FDF7CAF8002248F2F0117F48FDF7C4F86B
:1077940000224FF2E9317D48FDF7BEF800220421B2
:1077A4007B48FDF7B9F849F6F07308A975480893C2
:1077B4000B9609970A94FCF7BDFF764B08A971480C
:1077C400099308970A94FCF7B5FF48F2F01308A947
:1077D4006D4808930B9609970A94FCF7ABFF4FF298
:1077E400E93308A9694808930B9609970A94FCF7AA
:1077F400A1FF042308A9664808930B9609970A94E5
:10780400FCF798FF08A96148CDF8209009940A94E0
:10781400FCF790FF6B69604A3B436B616B694046C0
:107824003B400193019B40F23F6388E80C0009232D
:107834005A4EC8F80C3008940994C8F80840C8F89F
:107844001840FEF739F808A9404608940994FEF751
:107854004DF8534B534D304686E80808C6F814A03B
:10786400B460F4603461B461F461FEF737F94E4BEF
:10787400284685E80808C5F814A0AC60EC602C61C3
:10788400AC61EC61FEF72AF948484949494BDFF8F5
:1078940040A180E80A004FF4804384600361C4601F
:1078A40044618461C4610462FDF716FA424B504698
:1078B4008AE818004FF47A73CAF80830FDF742FCDE
:1078C400224621460F20FCF717FD0F20FCF748FD48
:1078D400224621462520FCF70FFD2520FCF740FD1C
:1078E400224621462620FCF707FD2620FCF738FD1A
:1078F400224621463620FCF7FFFC3620FCF730FDFB
:10790400224621464846FCF7F7FC4846FCF728FD8A
:10791400224621460620FCF7EFFC0620FCF720FD5A
:107924004046FDF7CBFE254B3A46254930461F70AD
:10793400FEF75EF93A4623492846FEF759F9224BE9
:1079440021461B68986800F09BFA9DF81A1006A857
:107954000331C9B2FFF784FBFFF786FE4CF6CC4235
:10796400DAF800301A60FEF78DFBFFF7D1FCFEF762
:10797400FFFDFFF709FDFFF765FDFFF7E1FDF6E702
:10798400001002400010014000080140000C0140BA
:107994000014014000001110001000402C070020CA
:1079A40000380140D8080020004400400C060020A4
:1079B40000580040A086010000300040010400206F
:1079C40034080020600600201400002098080020DD
:1079D40000060020704710B5FF230446221AD2B2D5
:1079E400914201D8184610BD14F8012B53400822C7
:1079F40013F0800F02F1FF324FEA430318BF83F004
:107A0400310312F0FF02DBB2F2D1E7E730B5FF2316
:107A140005462C1AE4B2A14203D89B1A5842584195
:107A240030BD15F8014B6340082413F0800F04F1B6
:107A3400FF344FEA430318BF83F0310314F0FF040B
:107A4400DBB2F2D1E5E700000E4B82B09A6942F056
:107A540001029A619A6902F001020092009ADA69BD
:107A640042F08052DA61DB69074A03F080530193E4
:107A7400019B536823F0E06343F00073536002B04A
:107A8400704700BF001002400000014010B50446DA
:107A940086B01022002102A800F06DF92268114B73
:107AA4009A421DD1104C02A9A369104843F008035F
:107AB400A361A36903F008030093009B4FF44063A0
:107AC40002931223039303230593FCF733FEE36924
:107AD40043F48003E361E36903F480030193019BAE
:107AE40006B010BD0058004000100240000C0140D8
:107AF4000268084B82B09A420AD103F50033DA696E
:107B040042F01002DA61DB6903F010030193019B78
:107B140002B0704700100040102270B5064688B0CD
:107B24000DEB0200002100F026F93368364A934237
:107B34003DD1364B04A99A69354842F480429A6192
:107B44009A69002502F480420092009A9A69314CA5
:107B540042F004029A619B6903F004030193019BC0
:107B64004FF4007304930223059303230793FCF754
:107B7400E1FD4FF4806304A9254804930595069517
:107B8400FCF7D8FD244B84E828008023E3602023FD
:107B9400A56025616561A361E5612046FCF702FCEF
:107BA40008B1FFF717FF7463666208B070BD1B4A23
:107BB4009342FAD1154B04A9DA69154842F400320C
:107BC400DA61DA69002502F400320292029A9A69B3
:107BD400134C42F004029A619B6903F0040303937B
:107BE400039B042304930223059303230793FCF7C5
:107BF400A1FD082304A90648049305950695FCF7FE
:107C040099FD084BBFE700BF003801400010024057
:107C140000080140E80600205800024000440040EB
:107C2400B40500206C0002407047FEE7FEE7FEE763
:107C3400FEE7704770477047FCF728BB0120FCF74C
:107C440075BE00000148FCF799BC00BFE80600209F
:107C54000148FCF793BC00BFB40500200148FEF7BF
:107C640099B800BF2C0700200148FEF793B800BF65
:107C7400D80800200148FDF730BD00BF9808002057
:107C84000E4B1A6842F001021A6059680C4A0A4005
:107C94005A601A6822F0847222F480321A601A68D8
:107CA40022F480221A605A6822F4FE025A604FF4C9
:107CB4001F029A60034A044B9A6070470010024006
:107CC4000000FFF80040000800ED00E0002103E0A0
:107CD4000B4B5B58435004310A480B4B42189A42F1
:107CE400F6D30A4A02E0002342F8043B084B9A42C6
:107CF400F9D3FFF7C5FF00F00FF8FFF7EFFC70476B
:107D0400789100080000002078000020780000200E
:107D1400340A0020FEE7000070B500250C4E0D4C1F
:107D2400A41BA410A54209D101F08AF800250A4E2B
:107D34000A4CA41BA410A54205D170BD56F82530E9
:107D440098470135EEE756F8253098470135F2E7B4
:107D540070910008709100087091000874910008F7
:107D640010B5431E0A44914200D110BD11F8014BD5
:107D740003F8014FF7E703460244934200D17047EA
:107D840003F8011BF9E700000FB40A4B13B51C6894
:107D940024B1A36913B9204600F0DAFA05AB049ABA
:107DA400A1682046019300F09BFC02B0BDE810409E
:107DB40004B070471400002070B50E46054618B193
:107DC40083690BB900F0C4FAAB69AC6813B92846EF
:107DD40000F0BEFA234B9C4217D16C68A3891B07A1
:107DE4001DD52369DBB1013EA36816F8011F013BD1
:107DF400A360E9B9002B2EDA22460A21284600F0B6
:107E0400F5F8013011D00A2070BD174B9C4201D106
:107E1400AC68E3E7154B9C4208BFEC68DEE72146FB
:107E2400284600F035F90028DDD04FF0FF3070BD52
:107E3400002B04DAA269934206DB0A2904D02368E2
:107E44005A1C22601970CFE72246284600F0CEF86B
:107E54000130C9D1E9E70A2023685A1C226018704E
:107E640070BD00BFFC9000081C910008DC90000865
:107E7400024B01461868FFF79FBF00BF14000020A3
:107E840000294FF480630CBF0222002200F000B8E6
:107E94002DE9F7431D46514B04461E680F46904694
:107EA40026B1B36913B9304600F052FA4C4B9C42E8
:107EB40052D17468B8F1020F06D0B8F1010F00F284
:107EC4008980002DC0F286802146304600F0D6F924
:107ED400616B41B104F14403994202D0304600F091
:107EE4002DFB002363630023A3616360A3891B0646
:107EF40003D52169304600F021FBA389B8F1020FB4
:107F040023F44A6323F00303A3815DD001AB6A46E3
:107F14002146304600F0A6FAA3891843A0812DBB60
:107F2400009D284600F002FB074600284ED1DDF8EC
:107F34000090A9453CD14FF0FF30A38943F00203E0
:107F4400A3810023A36004F1470323602361012379
:107F5400636103B0BDE8F083224B9C4201D1B46855
:107F6400A8E7214B9C4208BFF468A3E7002FD8D0B0
:107F7400B36913B9304600F0EBF9B8F1010F08BF4B
:107F8400A389276004BF43F00103A381A389276168
:107F940013F0080065611BD013F001004FF00003DB
:107FA4001FBF6D42A360A561184608BFA560D0E756
:107FB400484600F0BBFA07460028BCD0A3894D46CA
:107FC40043F08003A381D3E70020B6E7A946F5E791
:107FD400A060BEE74FF0FF30BBE700BF14000020F5
:107FE400FC9000081C910008DC900008F8B50E46CF
:107FF4001446054618B183690BB900F0A9F9214B61
:108004009C422AD16C68A369A360A3891A072ED560
:10801400236963B323692068F6B2C01A63693746DB
:10802400984204DB2146284600F028F928BBA368BF
:108034000130013BA36023685A1C22601E706369EF
:10804400984204D0A389DB0719D50A2E17D12146FB
:10805400284600F013F990B10FE00B4B9C4201D17C
:10806400AC68D0E7094B9C4208BFEC68CBE72146DB
:10807400284600F00DF80028CCD04FF0FF373846E2
:10808400F8BD00BFFC9000081C910008DC900008BB
:10809400324B70B51D6806460C4625B1AB6913B961
:1080A400284600F055F92E4B9C420FD16C68B4F968
:1080B4000C309AB215072CD4D00611D409223260A0
:1080C40043F04003A3814FF0FF3070BD254B9C4229
:1080D40001D1AC68EBE7244B9C4208BFEC68E6E7AF
:1080E400510712D5616B41B104F14403994202D0A6
:1080F400304600F023FA00236363A38923F02403AA
:10810400A3810023636023692360A38943F00803E8
:10811400A38123694BB9A38903F42073B3F5007FCA
:1081240003D02146304600F0C1F9A28912F00103C0
:108134000CD00023A36063695B42A361236953B934
:10814400B4F90C3013F08000BAD170BD920758BF57
:108154006369A360F2E70020F7E700BF1400002082
:10816400FC9000081C910008DC9000088A892DE925
:10817400F041054610070C465AD44B68002B05DC29
:108184000B6C002B02DC0020BDE8F081E66A002EB7
:10819400F9D0002312F480522F682B6033D0606D25
:1081A400A3895A0705D56368C01A636B0BB1236CA6
:1081B400C01A00230246E66A216A2846B047431CD7
:1081C400A38906D129681D294BD82B4ACA40D60752
:1081D40047D5002262602269D904226004D5421C7A
:1081E40001D12B6803B96065616B2F600029CAD087
:1081F40004F14403994202D0284600F09FF900207C
:108204006063BDE8F081216A01232846B047411C20
:10821400C6D12B68002BC3D01D2B01D0162B01D146
:108224002F60B0E7A38943F04003A381BDE8F08148
:108234000F69002FA7D0930718BF00230E6808BF4B
:108244004B69A6EB07080F608B60B8F1000F9ADD4D
:1082540043463A46216A2846A66AB047002807DC06
:10826400A38943F04003A3814FF0FF30BDE8F081C0
:108274000744A8EB0008E8E70100402038B50B6983
:1082840005460C46DBB118B183690BB900F060F800
:108294000C4B9C4209D16C68B4F90C307BB121467B
:1082A4002846BDE83840FFF761BF074B9C4201D127
:1082B400AC68F1E7054B9C4208BFEC68ECE7002092
:1082C40038BD00BFFC9000081C910008DC90000839
:1082D400014900F0A9B800BF81820008002310B54D
:1082E400044603604360836081814366C281036105
:1082F40043618361194608225C30FFF73CFD054B5E
:1083040024626362044BA362044BE362044B236361
:1083140010BD00BF618C0008838C0008BB8C000872
:10832400DF8C000870B568254A1E55430E4605F1DA
:10833400740100F04FF9044640B1002180E8420086
:108344000C30A06005F16802FFF715FD204670BDF2
:10835400836910B5044633BB8364C3640365124B5D
:10836400124A1B688262984204BF0123836100F0B1
:108374001FF86060204600F01BF8A060204600F063
:1083840017F80022E06004216068FFF7A7FF0122CC
:108394000921A068FFF7A2FF02221221E068FFF77B
:1083A4009DFF0123A36110BDD8900008D582000869
:1083B400F8B51C4B07461E68B36913B93046FFF77E
:1083C400C7FF4836B4687368013B03D5336833B1DB
:1083D4003668F7E7B4F90C506DB16834F4E704215A
:1083E4003846FFF79FFF30600028F1D10C23044684
:1083F4003B602046F8BD4FF6FF73E38101236566B9
:10840400A3812560A560656025616561A561082279
:10841400294604F15C00FFF7AEFC6563A563A5641F
:10842400E564E6E7D89000082DE9F84380468946DC
:10843400002600F1480414B93046BDE8F883A56865
:108444006768013F01D52468F5E7AB89012B07D99B
:10845400B5F90E30013303D029464046C8470643D8
:108464006835EEE770B50E46B1F90E1090B00029EC
:1084740014461D4607DA00232B60B3891A0610D46C
:108484004FF480630EE001AA00F04EFC0028F2DBFA
:10849400029A02F47042A2F500535A425A412A60E9
:1084A400EEE740230020236010B070BD8B8973B5C4
:1084B4009D0706460C4607D504F147032360236154
:1084C4000123636102B070BD01AB6A46FFF7CAFFC6
:1084D40000990546304600F07DF848B9B4F90C30EF
:1084E4009A05EFD423F0030343F00203A381E3E7E7
:1084F4000D4BB362A389206043F08003A381009BEA
:1085040020616361019B5BB1B4F90E10304600F049
:108514001DFC28B1A38923F0030343F00103A381C5
:10852400A3891D43A581CDE7D5820008024B0146EE
:10853400186800F04FB800BF1400002038B5054695
:10854400002943D051F8043C0C1F002BB8BFE41899
:1085540000F02CFC1E4A1368104633B963601460A3
:108564002846BDE8384000F022BCA3420BD921685C
:108574006218934201BF1A685B68521822606360F4
:108584000460EDE713465A680AB1A242FAD91968A1
:108594005818A0420BD1206801445818824219602F
:1085A400DED110685268014419605A60D8E702D9D4
:1085B4000C232B60D4E7206821188A4201BF11687C
:1085C40052680918216062605C60C9E738BD00BF69
:1085D400A405002070B5CD1C25F0030508350C2D2D
:1085E40038BF0C25002D064601DBA94203D90C2314
:1085F4003360002070BD00F0D9FB234A1468214683
:1086040091B9224C23681BB9304600F017FB206057
:108614002946304600F012FB431C26D10C23304679
:10862400336000F0C4FBE4E70B685B1B1AD40B2B2C
:108634000FD90B60CC18CD50304600F0B8FB04F1D4
:108644000B00231D20F00700C31A1BD05A42E2502E
:1086540070BD8C420BBF63684B681360636018BFC6
:108664000C46E9E70C464968CAE7C41C24F0030435
:10867400A04205D0211A304600F0E0FA0130CDD0F6
:108684002560D9E770BD00BFA4050020A80500201F
:10869400936810B4013B002B936008DA9469A342F9
:1086A40002DBCBB20A2B02D110BCFFF79FBC1368CC
:1086B400581C10601970C8B210BC7047F8B5064653
:1086C4000F461446D518AC4201D1002007E03A46C3
:1086D40014F8011B3046FFF7DBFF431CF3D1F8BD50
:1086E4002DE9F04F9DB00C4617460393064618B18A
:1086F40083690BB9FFF72CFE7C4B9C4257D17468FD
:10870400A38918075DD52369002B5AD00023099348
:1087140020238DF8293030234FF0010B8DF82A30B7
:10872400B846454615F8013B002B55D1B8EB070A6E
:108734000BD053463A4621463046FFF7BFFF01307F
:1087440000F0C480099B5344099398F80030002B2F
:1087540000F0BC8000234FF0FF320493079305928E
:1087640006938DF853301A9305222978604800F057
:108774000FFB05F10108049B002831D1D90644BF41
:1087840020228DF853201A0744BF2B228DF8532042
:108794002A782A2A2CD000210A20079AA84698F879
:1087A40000300135303B092B6DD971B326E0514BB4
:1087B4009C4201D1B468A3E74F4B9C4208BFF468C4
:1087C4009EE721463046FFF763FC00289ED04FF019
:1087D400FF301DB0BDE8F08F252BA7D0A846A0E739
:1087E400434A4546801A0BFA00F018430490BBE74D
:1087F400039A111D12680391002A01DB079204E019
:10880400524243F002030792049398F800302E2B4F
:1088140010D198F8013008F101012A2B37D1039BBC
:1088240008F102081A1D1B680392002BB8BF4FF011
:10883400FF330593314D032298F80010284600F0C9
:10884400A7FA40B14023401B03FA00F0049B08F14F
:1088540001080343049398F800100622284808F1FD
:1088640001078DF8281000F093FA002834D0254B26
:1088740003BB039B073323F0070308330393099BCC
:108884004B4409934CE700FB0232012186E70023A5
:108894000A2518460593884698F800200131303A95
:1088A400092A03D9002BC5D00590C3E705FB002096
:1088B4000123F0E703AB00932246134B04A930468F
:1088C400AFF30080B0F1FF3F8146D8D1A3895B06A6
:1088D4003FF57DAF09987CE703AB009322460A4B32
:1088E40004A9304600F08AF8ECE700BFFC900008C9
:1088F4003C9100081C910008DC900008429100089B
:108904004691000800000000C18600082DE9F047E8
:1089140091461F468A680B6906469342B8BF1346C0
:10892400C9F8003091F843200C46DDF8208012B1DC
:108934000133C9F800302368990642BFD9F80030E2
:108944000233C9F80030256815F0060507D104F193
:10895400190AE368D9F800209B1A9D422ADB94F88F
:1089640043302268003318BF012392062FD404F148
:10897400430239463046C047013022D02368E568B7
:1089840003F00603042B18BF0025D9F800204FF08C
:10899400000908BFAD1AA368226908BF25EAE57576
:1089A4009342C4BF9B1AED181A344D451BD10020C5
:1089B400BDE8F0870123524639463046C0470130AE
:1089C40003D14FF0FF30BDE8F0870135C1E7302017
:1089D400E11881F843005A1C94F8451022440233EC
:1089E40082F84310C3E70123224639463046C04784
:1089F4000130E6D009F10109D7E700002DE9F04381
:108A040017460A7E85B06E2A984606460C460C9B8D
:108A140001F1430E00F0BC801AD8632A2ED00AD884
:108A2400002A00F0C880582A00F08A8004F1420528
:108A340084F842202AE0642A01D0692AF6D1216808
:108A44001A6811F0800F23D0111D1960136827E0F4
:108A5400732A00F0B48008D86F2A2AD0702AE5D18E
:108A64000A6842F020020A6003E0752A21D0782ABD
:108A7400DCD178226F4984F8452064E01A6801F15A
:108A84004205111D1960136884F842300123A3E0E4
:108A940011F0400F02F104011960D7D0B2F900308F
:108AA400002B03DA2D225B4284F8432062490A2218
:108AB40017E02068196810F0800F03D0081D1860B3
:108AC4000B6806E010F0400F01F104001860F7D0C5
:108AD4000B886F2A14BF0A2208225749002084F801
:108AE40043006568002DA560C0F29C80206820F0DA
:108AF40004002060002B3FD1002D40F09580754686
:108B0400082A0BD12368DA0708D5236962689A42D8
:108B1400DEBF302305F8013C05F1FF35AEEB05035C
:108B24002361CDF800803B4603AA21463046FFF777
:108B3400EDFE013055D14FF0FF3005B0BDE8F083B4
:108B440081F845203C492268186812F0800F00F132
:108B540004051D6001D0036802E05506FBD50388B7
:108B6400D00744BF42F0200222601BB9226822F0E1
:108B7400200222601022B1E77546B3FBF2F002FB3B
:108B84001033CB5C05F8013D03460028F5D1B7E767
:108B940008681A6810F0800F496904D0101D186025
:108BA4001368196007E010F0400F02F10400186028
:108BB4001368F6D01980002375462361B1E71A685B
:108BC400111D1960156800216268284600F0E0F85C
:108BD40008B1401B606063682361002384F843305C
:108BE4009FE723692A4639463046C0470130A2D060
:108BF40023689B0707D5002504F11909E368039A44
:108C04009B1A9D4205DBE068039B9842B8BF184657
:108C140093E701234A4639463046C04701308AD09B
:108C24000135EBE7002BA7D10B7804F1420584F85A
:108C3400423065E75E9100084D91000838B5002385
:108C4400054C05460846236000F0ECF8431C02D1AD
:108C5400236803B12B6038BD300A002010B50C46E0
:108C6400B1F90E1000F0A4F80028ABBF636DA3891E
:108C74001B1823F48053ACBF6365A38110BD2DE999
:108C8400F0411F468B890546DB050C46164605D583
:108C940002230022B1F90E1000F068F8A3893246CD
:108CA40023F48053A381B4F90E103B462846BDE853
:108CB400F04100F017B810B50C46B1F90E1000F0F1
:108CC40055F8431CA38915BF606523F4805343F40E
:108CD4008053A38118BFA38110BDB1F90E1000F019
:108CE40013B8000038B50546084611460022054C65
:108CF40022601A46FEF7BCF9431C02D1236803B173
:108D04002B6038BD300A002038B50023054C0546D9
:108D14000846236000F05EF8431C02D1236803B1C7
:108D24002B6038BD300A002038B50023064C0546B8
:108D340008461146236000F055F8431C02D123680D
:108D440003B12B6038BD00BF300A002038B50023C2
:108D5400054C05460846236000F04CF8431C02D13C
:108D6400236803B12B6038BD300A002038B50546AE
:108D7400084611460022054C22601A4600F042F8CB
:108D8400431C02D1236803B12B6038BD300A002094
:108D940010B5C9B202449042034601D1002010BD6F
:108DA4001C7801308C42F6D1184610BD70477047CC
:108DB40038B50546084611460022054C22601A467D
:108DC40000F028F8431C02D1236803B12B6038BD9E
:108DD400300A00205822024B4FF0FF301A607047CF
:108DE400300A00205822024B4FF0FF301A607047BF
:108DF400300A00205822024B00201A60704700BF3E
:108E0400300A00205822024B4FF0FF301A6070479E
:108E1400300A00205822024B4FF0FF301A6070478E
:108E2400300A0020044B0246196809B90349196045
:108E3400186802441A607047AC050020340A002008
:108E4400F8B500BFF8BC08BC9E467047F8B500BF33
:088E5400F8BC08BC9E46704703
:108E5C0002030405060708090A0B0C0D0E0F10106F
:108E6C00454550524F4D2053415645204552524F87
:108E7C0052212121200001070D13191F252B32002F
:108E8C0064009600C800FA002C015E0190010407F2
:108E9C000A0D101D20235265636F676E697A652079
:108EAC0025642053656E736F720A004D59206964F6
:108EBC00206973202564200A005247425F53656E77
:108ECC00736F725265644C696D69745F4275665B51
:108EDC0025645D202020203A2020253034780A009B
:108EEC005247425F53656E736F72477265656E4C85
:108EFC00696D69745F4275665B25645D20203A205C
:108F0C0020253034780A005247425F53656E736FE8
:108F1C0072426C75654C696D69745F4275665B2550
:108F2C00645D2020203A2020253034780A004C6FD4
:108F3C007261206672657175656E637920202020E0
:108F4C00203A202564200A004C6F7261204C6F522D
:108F5C00615F50615F626F6F7374203A20256420EB
:108F6C000A004C6F7261204C6F52615F52617465E4
:108F7C0020202020203A202564200A004C6F7261AA
:108F8C00204C6F52615F4257202020202020203A35
:108F9C00202564200A004C6F7261204C6F52615F77
:108FAC004C6E612020202020203A202564200A00CD
:108FBC004E6F7420457869737420446576696365D7
:108FCC002000E54026E56026E58026E5A026E5C0E4
:108FDC0026E5E026E60026E62026E64026E6602684
:108FEC00E68026E6A026E6C026E6E026000102037F
:108FFC0004050607080946756E6374696F6E203A9E
:10900C00202573202020204C696E65203A20256491
:10901C00200A00FFFCF9F6060708090A0B0C535846
:10902C00313237365F4C6F5261456E7472795278BB
:10903C00005358313237365F4C6F5261456E747243
:10904C00795478005358313237365F4C6F52615433
:10905C00785061636B65740052737369203A2025F4
:10906C0064200A002530327820004F726967696EDF
:10907C00616C20435243203A2025303278205265CF
:10908C006376435243203A2025303278200D0A0073
:10909C00576861742048617070656E3F0D004920FF
:1090AC00616D20526573657420466C616720436C5A
:1090BC006561720000000000000000000102030462
:1090CC000607080900000000010203041800002034
:1090DC000000000000000000000000000000000084
:1090EC000000000000000000000000000000000074
:1090FC000000000000000000000000000000000064
:10910C000000000000000000000000000000000053
:10911C000000000000000000000000000000000043
:10912C000000000000000000000000000000000033
:10913C00232D302B2000686C4C0065666745464734
:10914C0000303132333435363738394142434445B7
:10915C004600303132333435363738396162636426
:04916C006566000034
:0491700009420008A8
:04917400E5410008C9
:109178000100000010000000000102030A010000C5
:1091880000A24A041800002000000000FC9000081B
:109198001C910008DC90000800000000000000009E
:1091A80000000000000000000000000000000000B7
:1091B80000000000000000000000000000000000A7
:1091C8000000000000000000000000000000000097
:1091D8000000000000000000000000000000000087
:0891E80000000000000000007F
:0400000508007CD1A2
:00000001FF
